:1000000002C700001CC700000C94311518C700007F
:1000100016C700000C94AB1812C7000010C70000F0
:100020000EC700000C943C1D0AC7000008C7000062
:1000300006C7000004C7000002C7000000C7000098
:10004000FEC60000FCC60000FAC60000F8C60000AC
:10005000F6C600000C94431FF2C60000F0C6000074
:10006000EEC60000ECC60000C00000000000B600B4
:10007000D608D008C600C1084A08CF009A0733083E
:10008000D500A7079B08E500AF077508F200B70782
:1000900042080001BF075E080901CC0724081601C9
:1000A000DB0752082601E80715083201F6070608A3
:1000B000000000000000456967656E652049440046
:1000C0005345545550004B6F6E7472617374004CFD
:1000D00069636874005369676E616C3A204D65739B
:1000E00073616765005369676E616C3A205573658B
:1000F000720053656E64657665727375636865003A
:100100004672657175656E7A00435120656D706643
:10011000616E67656E0042616B656E20496E746545
:100120007276616C6C005265706561742D466C610D
:1001300067004645430048415550544D454E5500D3
:100140004D48656172640056657266617373656ED1
:10015000004E6163687269636874656E004572770A
:1001600065697465727400536574757000417573C8
:10017000736368616C74656E0036010000000040B6
:1001800001DB0900004701BD0900005101B9090068
:10019000005D01AC0900006701B20900006D016D4E
:1001A000090000000000000000DD0100000000E781
:1001B000011B0A0000D301FC090000EE01E909005F
:1001C000000002E00900000C02DE0900000000004F
:1001D000000000456D7066E46E676572005645521A
:1001E00046415353454E0053656E64656E00456E3F
:1001F00074777572662073706569636865726E00E6
:1002000054657874206C656572656E004265656E34
:1002100064656E0044657461696C73005D02000082
:10022000000046027E0A000050026E0A00006702CB
:10023000620A00007502670A00001402640A0000E6
:10024000000000000000416E74776F7274656E00EC
:100250005765697465726C656974656E004E4143DB
:100260004852494348540045726E65757420736561
:100270006E64656E004CF6736368656E0053656E60
:1002800064656E009C02000000007D029B0A000075
:10029000A3029D0A00000000000000004D484541F7
:1002A0005244004C69737465206C656572656E001C
:1002B000000108080900213C221F243E21322A2582
:1002C000222A150C083F2E2A131C2A11023A0F1459
:1002D0002A15042A1D290814232214093C0A3D3E2C
:1002E0002A151C22233E221D3E2A233E0A031C22DD
:1002F0003B3E083F223E2310201F3E08373E202170
:100300003E0C3F3E043F1C221D3E0A051C323D3E72
:100310000A352C2A1B023E033E203F1E201F3E189A
:100320003F360837063807322A2732283B000001BB
:10033000BEBF0E000E0128FE2828FE294C9EF29E0C
:10034000F2650C12522C10689490616CFE92BE6C97
:10035000E0990403387CC68382C67C3914083E08C1
:100360001508083E08093071101011C0C1C0300FC7
:100370007CFE8282FE7D84FEFE818CC2E2B29E8D76
:1003800044829292FE6D302824FEFE214E8E8A8A8F
:10039000FA737CFE9292F2610202E2FA1E076CFE90
:1003A0009292FE6D0C9E92D27E3DEC0D6C6D3030C3
:1003B00048488485282828282984844848303104DE
:1003C000A2B21E0D384492BAAA9ABA2419E0F83E95
:1003D000263EF8E1FEFE9292FE6D7CFE8282C645CC
:1003E000FEFE8282FE7DFEFE929283FEFE121203CC
:1003F0007CFE8292F2F5FEFE101010FEFF82FEFEE1
:10040000838082FE7FFEFE386CC683FEFE80808184
:10041000FEFE0E1C38180CFEFFFE0E1C3870FF7C12
:10042000FE828282FE7DFEFE22223E1D3C7E4262D4
:10043000C2FEBDFEFE3272DE8D4C9EBAF265020235
:10044000FEFE02037EFE8080FE7F0E3EF0F03E0F39
:100450003EFEC03E3EC0FE3FC6EE3838EEC7061E2A
:10046000F8F81E07E2F2BA9E8FFEFE82830638C1BC
:100470008282FEFF0804020204098080808080815D
:10048000020540E8A8F8F1FEFE88F87170F8888946
:1004900070F888FEFF70F8A8B8B1FCFE0A0310B827
:1004A000A8F879FEFE08F8F1FAFB88FA7BFEFE70E8
:1004B000D889FEFFF8F808F8F008F8F1F8F808F81D
:1004C000F170F888F871F8F8283811103828F8F920
:1004D000F8F8101990B8E8497CFC8978F880F8F9A8
:1004E0001878E0781938F8C030C0F839D8F820F812
:1004F000D918B8E07819C8E8B899E3F83E263EF86C
:10050000E77AFE848484FE7B7AFA8080FA7B42EA72
:10051000A8FAF372FA88FA737AFA80FAFBFC7E92F0
:10052000FE6D000001BF0E000F20E83E28F82E09E6
:100530008894FEA4454626100864636C92926C5021
:100540008104020138448382443914083E081508A6
:10055000083E0809C1202141C038077C82827D8481
:10056000FE81C2A2928D8292926D302824FE219E3D
:100570009292637C92926182621A076C92926D0CE5
:1005800092927D8069D920505050895050505050DF
:1005900051885050502102A2120D384492AABA2418
:1005A00019E0382638E1FE92926D7C82828245FE07
:1005B00082824439FE929283FE1212037C829292CE
:1005C000F5FE10101010FF82FE8380827FFE10283F
:1005D0004483FE808081FE0618601806FFFE040832
:1005E0001020FF38448282824439FE2222221D38A4
:1005F0004482A242C4B9FE1232528D8C929292630E
:100600000202FE02037E808080807F0E30C0C030F8
:100610000F3EC0380638C03FC6281028C70618E06D
:100620001807C2B28A87FE830638C182FF08040217
:1006300004098080808081020540A8A8F1FE888896
:1006400071708889708888FF70A8A8B1FC12131097
:10065000A8A879FE0808F1FB887BFE205089FFF8E6
:100660000808F00808F1F80808F170888871F8287F
:100670002811102828F9F8100990A8497C89788059
:1006800080F9186080601938C0601860C039D820BF
:10069000D918A0A079C8A899E2382638E33A44824C
:1006A0008282443B7A808080807B40AAA8F3728853
:1006B00088737A8080FBFC02926D2D032205B002C4
:1006C0003003250500003203260500003603290506
:1006D00000003C03300500004203350500004B03D9
:1006E0003B0500005203410500005403440500008F
:1006F0005803470500005C034A05000061034F05ED
:10070000000066035405000068035505B2026B0340
:100710005705B5026D035805000070035B05B7026D
:1007200076035F05BA027A036205BD02800366059F
:10073000C00286036A05C3028C036F05C6029203DA
:100740007305C90298037705CC029E037B05CF028F
:10075000A4037F05D202AC038505D502AA03830555
:100760000000AE038605D602B4038B050000B90372
:100770009105D902BF0396050000C4039A05000045
:10078000CD03A105DC02D403A605DF02DA03AA0526
:10079000E202E003AF05E502E603B405E802EB037D
:1007A000B805EB02F003BC05EE02F603C105F10249
:1007B000FD03C705F4020104CA05F7020504CD05CF
:1007C000FA020B04D205FD021004D6050003190439
:1007D000DD0503031F04E30506032604EA050903F8
:1007E0002C04EF050C033304F6050F033904FB0555
:1007F00012033E04000615034404050618034A04C8
:100800000B061B03500411061E035804180621038F
:100810005E041D06240364042206270369042606D9
:1008200000006D042806000070042B06000074040C
:100830002D0600007A04320600008004370600000E
:1008400082043906DC0287043D06DF028C0441067F
:10085000E20290044406E50295044806E8029A0480
:100860004C06EB029E044F06EE02A3045306F1026F
:10087000A8045706F402AA045806F702AD045A0663
:10088000FA02B2045E06FD02B4045F060003BC0473
:1008900066060303C1046A060603C6046E0609035E
:1008A000CB0472060C03D00476060F03D404790639
:1008B0001203D8047C061503DB047E061803E0044B
:1008C00082061B03E50487061E03EC048E06210343
:1008D000F10491062403F60495062703FA0498060A
:1008E0002A0301059D0600000805A40600000E0568
:1008F000AA062A031305AE0600001805B20600007A
:100900001D05B60600008A0996097E0970092E2C7D
:100910003F2127222D2829402F3A5F3B2B26252ACD
:100920003D3C3E40245B5D5C5E60AAAA2DD4AAAA31
:10093000AA2DD4AA2DD4AA2DD4AA2DD4AAF0CC3372
:100940005A4351005549003337350041756720320D
:100950003320323030390031353A31393A313700CD
:10096000204765727269742044483847484800003F
:100970000D102844002844824428004428100B24E9
:100980003E2000322A2400222A140B302838003E50
:100990002810001028280B3C0A3C003E2A14001C9A
:1009A000222207E08890A09088E007E08890AE902F
:1009B00088E007E08884BA8488E007E0868ABE8AF7
:1009C00086E007E080A8A8A880E007E080A890A8BB
:1009D00080E00503053F0503087F4345494945433A
:1009E0007F081C2214001C223C2046694669534D96
:1009F00053657200417573736368616C74656E2032
:100A00003F004E4F43414C4C004E61636872696336
:100A10006874656E0045696E74726167206CF67368
:100A20006368656E3F006D696E004E6F742073657C
:100A300065206D65004D48204C6973746500446500
:100A40007461696C7300416273203A2000456D70D7
:100A5000663A20005A6569743A004B65696E204514
:100A60006D7066E46E6765722067657365747A748D
:100A70002E20416E20616C6C652073656E64656E1E
:100A8000203F00435100416E736568656E006175DB
:100A9000730065696E004D736720696E20506F7337
:100AA000746175732D2067616E672065696E676577
:100AB0007265696874004D657373616765656E740E
:100AC00077757266206162676573706569636865D2
:100AD000727400454E545755524600537065696311
:100AE00068657220766F6C6C21204E696368742093
:100AF000676573706569636865727400416C6C65E5
:100B0000204E6163687269636874656E206CF67369
:100B10006368656E203F004B616C7473746172741E
:100B20002064757263682D2066FC6872656E3F00F4
:100B30004265657000566962726100426565702F9A
:100B4000566962726100204F4B2000204241434BA6
:100B50002000204A612000204E65696E2000203C64
:100B60002D2000205345542000204D454E55452052
:100B700000204D482000204D534720003C2D2000F0
:100B80002D3E20003433342E353030003433392EAE
:100B9000373030003433342E39303000D80B06066D
:100BA000DA0B3703E10B3812E70B390CED0B330B83
:100BB000F20B3211F80B310200000000020C151587
:100BC000040C2A2A060C301B090C23230B0C3613A9
:100BD000110C350A160C341406007071727337DF6D
:100BE0000074757638FC007778797A390064656628
:100BF000330061626332E4002E2C3F2131272D2F18
:100C00003A0015002A0020300023006D6E6F36F682
:100C1000006A6B6C35006768693400554900010251
:100C2000040810204080B10C00000000BB0C0A2218
:100C30000000CC0C25210000500CAC210000D90C88
:100C400098210000580C272100000000000000003F
:100C500056657273696F6E0048462D5465737466ED
:100C6000756E6B74696F6E00303A204144432D57A6
:100C700065727400333A205458206D6974205041D5
:100C800000323A20525800313A205458206F686E92
:100C900065205041004154004259005645520053CE
:100CA0005045494348455242454C4547554E4720DB
:100CB0000045525745495445525400537065696385
:100CC00068657262656C6567756E67004C6976650C
:100CD0002D6D6F6E69746F72004E657573746172FD
:100CE0007400000000000000000000000000000090
:100CF0000000000102030405060708090A0B0C0D99
:100D00000E0F00020406080A0C0E030107050B096A
:100D10000F0D000306050C0F0A090B080D0E070442
:100D200001020004080C03070B0F06020E0A05015E
:100D30000D0900050A0F07020D080E0B0401090C2E
:100D4000030600060C0A0B0D07010503090F0E0828
:100D5000020400070E090F0801060D0A030402052C
:100D60000C0B0008030B060E050D0C040F070A02FE
:100D7000090100090108020B030A040D050C060F06
:100D8000070E000A070D0E0409030F050802010BE8
:100D9000060C000B050E0A010F04070C02090D06D4
:100DA0000803000C0B0705090E020A06010D0F03CC
:100DB0000408000D0904010C0805020F0B06030EC0
:100DC0000A07000E0F010D03020C09070608040AAA
:100DD0000B05000F0D020906040B010E0C0308079A
:100DE000050AFF0001040208050A030E0907060DA3
:100DF0000B0C0102040803060C0B050A070E0F0D6D
:100E00000901F0CC335A11241FBECFEFD8E0DEBF6A
:100E1000CDBF11E0A0E0B1E0ECE4F9E502C005903F
:100E20000D92AA30B107D9F715E0AAE0B1E001C0F0
:100E30001D92A233B107E1F719D00C94A42CE0C89D
:100E400087E187B980E188B984EF8AB98FEF8BB9E0
:100E50008EE284B985E085B981E58CBD81E08DBDE8
:100E600083E08093640080936D00089514BE88E150
:100E70000FB6F89480936000109260000FBEE0DF20
:100E80000E94BC1AD3D178940E9487180E949818A7
:100E90000E94301F0E94AB1A0E94D2190E94E214D5
:100EA0000E94C7190E942A198A9741F48CEF9AE090
:100EB00060E00ED4882311F00E9405210E94FC1CE2
:100EC0000E94031F0E94D4208AB580618ABD0E94BF
:100ED000D2130E947F1935D38091C9029091CA0222
:100EE0008038910541F40AB403FE03C00E946212E7
:100EF00002C00E94D00F8091C9029091CA02805016
:100F0000904829F789E791E061E002D5E0CFF999AF
:100F1000FECF92BD81BDF89A80B50895F999FECFB4
:100F20001FBA92BD81BD60BD0FB6F894FA9AF99AC6
:100F30000FBE08958091520190E080FF91E0809172
:100F400052018E7F892B8093520180E00895809119
:100F500054018F5F83708093540180E008958091E5
:100F600055018F5F83708093550180E008958091D3
:100F700056018F5F87708093560180E008958091BD
:100F800053018F5F8093530180915301833010F0A0
:100F90001092530180E008958091520190E082FF09
:100FA00091E0990F990F809152018B7F892B80934B
:100FB000520180E00895809157018F5F809357011F
:100FC000809157018B3010F01092570180E0089506
:100FD0008091520190E081FF91E0990F8091520140
:100FE0008D7F892B8093520180E00895809152017A
:100FF00090E083FF91E0990F990F990F8091520132
:10100000877F892B8093520180E008959C01809115
:10101000520183FF05C0C90162E97AE00C94652B97
:10102000C9016EE87AE00C94652B9C018091520115
:1010300081FF05C0C90162E57BE00C94652BC90105
:1010400067E57BE00C94652B9C018091520182FF47
:1010500005C0C90162E57BE00C94652BC90167E519
:101060007BE00C94652B9C018091520180FF05C0B0
:10107000C90162E97AE00C94652BC9016EE87AE057
:101080000C94652BBC018091560190E04AE050E041
:101090000C94ED2BBC018091510190E04AE050E0AE
:1010A0000C94ED2BBC018091570190E04AE050E098
:1010B0000E94ED2B66E27AE00C945A2B9C01809101
:1010C0005301882321F4C90164E87BE007C08091C3
:1010D0005301813029F4C9016CE87BE00C945A2B50
:1010E000C90164E97BE00C945A2B9C018091550165
:1010F000882321F4C9016EE87AE00FC08091550180
:10110000813021F4C90160E37BE007C08091550183
:10111000823029F4C90165E37BE00C945A2B80915D
:101120005501833019F080E090E00895C9016BE328
:101130007BE00C945A2B9C0180915401882321F46C
:10114000C9016EE87AE00FC080915401813021F42A
:10115000C90160E37BE007C080915401823029F42B
:10116000C90165E37BE00C945A2B809154018330D4
:1011700019F080E090E00895C9016BE37BE00C94E6
:101180005A2B809151018E5F8093510180915101C2
:10119000893210F0109251010E94D21980E0089516
:1011A00069E471E048E050E00C94AA2BCF93DF9300
:1011B000CEE5D1E08FE0FE0111928A95E9F7CE01EC
:1011C00069E471E048E050E00E94AA2BCE0168E09B
:1011D00046EB50E020E0CDD4882339F089E491E05B
:1011E000BE0148E050E00E94AA2B80E0DF91CF9141
:1011F000089580915801855980936600F999FECF32
:1012000080E090E069E471E040E150E02EE837E0F2
:101210000E94D32B0E942C15882331F078940E94D1
:101220002C158823E1F7F8940C94E214CF93DF9304
:10123000F999FECF89E491E060E070E040E150E090
:1012400027E837E00E94B92BF999FECFC0E1D0E042
:10125000D2BDC1BDF89A80B58A3209F43BC081E0A5
:10126000809357018BE280935101809152018160FC
:1012700080935201109253018091520182608093B9
:10128000520183E08093560110925401109255014F
:1012900089E491E062E07AE048E050E00E946C2B43
:1012A000F999FECF80E090E069E471E040E150E020
:1012B0002EE837E00E94D32BF999FECFF999FECFA3
:1012C0001FBAD2BDC1BD8AE280BD0FB6F894FA9AAA
:1012D000F99A0FBEDF91CF9108951F9384EF99E0A3
:1012E00060E0F6D18823A9F11FB7F8948AB58F7E04
:1012F0008ABD8AB58F7D8ABD10928B0010928A00BC
:1013000010928900109288000E94C71984E20E94FE
:10131000BA1980E092E80E9473148BEA809364000B
:1013200084E00E94FB1C1FBF83B7817F866083BF60
:1013300083B7816083BF889583B78E7F83BF0AB4EC
:1013400004FEF2CF83E8809364000E94D2190E94C9
:10135000E21481E01F91089586E29CE061E0D8D21A
:1013600080E0089588E690E060E0D2D242DF80E03D
:1013700008950E94621280E00895EFECF2E08AEA9C
:10138000DF011D928A95E9F78091E102887F8360F1
:101390008093E10290915201929590728F7D892BFA
:1013A0008093E102CF01449666E947E451E021E0F1
:1013B000E0D380E00895F4D581E0089582E00895B7
:1013C00086E9E3EEF2E0DF011D928A95E9F781E01C
:1013D00008958091E102887F81608093E1020E94FC
:1013E000A91C882319F086EB9AE002C08BED9AE0E5
:1013F00061E06ED181E00895CF93DF93CEE5D1E037
:101400008FE0FE0111928A95E9F7CE016FEC72E050
:101410000E948B2BCE0168E043ED51E020E0A9D380
:10142000882329F08FEC92E0BE010E948B2B80E094
:10143000DF91CF910895CF93DF93EFECF2E001902D
:101440000020E9F73197EF5CF240329708F4D4DFDF
:10145000CFECD2E0FE0101900020E9F73197EC1BC0
:10146000FD0B329758F48AE59AE060E031D1882389
:1014700029F1CE0163E87AE00E94652B8091E102B8
:10148000887F83608093E1029091520192959072DF
:101490008F7D892B8093E1020E94A91C882319F07B
:1014A00086E99AE002C08BED9AE061E011D188E014
:1014B000EFECF2E0DF011D928A95E9F781E0DF9120
:1014C000CF91089583E008958AD080E0089585E162
:1014D0009AE060E0FDD0811182E00895EFECF2E047
:1014E00088E0DF011D928A95E9F7CF01449666E90D
:1014F00040E552E021E03DD381E008950F931F9332
:101500000FEC12E0C801085F1F4FB80148E050E03F
:101510000E94AA2B045F1F4F86E9F80111928A9559
:10152000E9F7C80166E946E452E021E022D381E010
:101530001F910F91089582E008950E94031F81E09A
:1015400008950AB401FE08C080E060E00E94BE1960
:1015500082ED99E00E94931A0AB403FE08C087E066
:1015600060E00E94BE1988ED99E00C94931A0895EA
:101570000F931F93CF93DF938C01EB0180E065E025
:101580000E94BE1982E06EE70E94A719011511059D
:1015900019F0C8010E94481A84E265E00E94BE1951
:1015A0008091CC02E82FF0E0EE0FFF1FEA5FF64FCC
:1015B000859194910E94931A209761F0CE010E9428
:1015C000711A94E5981B892F65E00E94BE19CE011F
:1015D0000E94481ADF91CF911F910F910895FF92B9
:1015E0000F931F930E94C719ACDF89E160E00E944E
:1015F000BE1982E060E80E94A71984E192E00E948F
:10160000481A86E49BE06BE47BE0B2DF81E060E0B7
:101610000E94A71980E061E00E94BE1986E49AE06A
:101620000E94481A0EE511E09FE0F92EF8012F2DD7
:1016300011922A95E9F7C80167ED72E048E050E0A1
:101640000E94AA2BC8010E94551A80E062E00E9405
:10165000BE198DE49AE00E94481AF8012F2D1192CC
:101660002A95E9F7C8016FEC72E048E050E00E946B
:10167000AA2BC8010E94551A80E063E00E94BE199F
:1016800084E59AE00E94481AF8011192FA94E9F769
:101690008091DF029091E002B8014AE050E00E94A0
:1016A000ED2B0E94551A0E947F198091C9029091DA
:1016B000CA028050904839F08091C9029091CA02C4
:1016C0008038910581F781E01F910F91FF90089577
:1016D000FF920F931F938C01F62E0E94C71980E092
:1016E00062E00E94BE1980E060E00E94A719C80174
:1016F0000E94481AFF2029F086E49BE060E070E039
:1017000004C082E59BE067E57BE032DF0E947F1941
:101710008091C9029091CA028050904811F481E0F2
:1017200008C08091C9029091CA028038910571F772
:1017300080E01F910F91FF900895EF92FF920F9319
:101740001F93CF93DF93962F682F70E088E2989FC6
:10175000C00111240E94302C22E0E22EE60E00E0AF
:10176000FF24C1E0D0E081E56F2D0E94BE1987E023
:101770008E15A8F0002399F48E010E2C02C0000FE4
:10178000111F0A94E2F7802F0E94BC19802F0E943B
:10179000BC19802F8A6A0E94BC1901E00BC080E04E
:1017A0000E94BC1980E00E94BC198AEA0E94BC1900
:1017B00088EFE80EF39486E0F816A9F6DF91CF9152
:1017C0001F910F91FF90EF900895AF92BF92CF922B
:1017D000DF92EF92FF920F931F93A090CC0283E0D1
:1017E0008093CC0210E0BB2403C01BE101C010E0D9
:1017F0000E94C719A6DE86E49BE06BE47BE0B8DEBE
:10180000EE24DD2428C0EF2DF0E0E25FF64FC49017
:101810001F1531F481E06FEF0E94A719BC2C04C0A2
:1018200081E060E00E94A719802F6E2D0E94BE19F2
:1018300080E20E942C1A8C2D0E942C1A80E20E94B9
:101840002C1AF394055F0D34F1F6E39487E0D80E7B
:1018500084E0E81619F0FD2C00E0D5CF0E947F1936
:101860008091C9029091CA020E94C0188C3009F47C
:10187000BCCF8D3088F48630D9F1873038F482308F
:1018800009F4B5CF833009F0B3CF30C08A3081F18D
:101890008B3009F0ADCF10C08331A9F0843130F422
:1018A0008131F1F0823109F0A3CF12C0843131F0DF
:1018B000853109F09DCF1FC016E09ACF112309F49E
:1018C00094CF115095CF1B3108F091CF1F5F90CF6F
:1018D000195F1C3108F48CCF17501830E8F788CF07
:1018E000173010F41B5E84CF175082CF15E180CFE4
:1018F000A092CC0203C0A092CC02BB248B2D1F91DE
:101900000F91FF90EF90DF90CF90BF90AF90089530
:101910002F923F924F925F926F927F928F929F92FF
:10192000AF92BF92CF92DF92EF92FF920F931F93ED
:10193000DF93CF9300D000D00F92CDB7DEB74C012C
:101940006983552436E0252D2F5F239FF001112454
:10195000E80DF91D85919491892B11F0522EF3CF4A
:1019600044244394BB24B394F401859194919B83C4
:101970008A83252C332493E09093CC020E94C719CC
:10198000E0DD89E160E00E94BE1982E060E80E942B
:10199000A7198A819B810E94481AAB2CAA94852D95
:1019A0006A2DCBDEA981AA2309F039C083E69BE02A
:1019B0006BE47BE0DDDD80E060E00E94A71980E061
:1019C00062E00E94BE19B6E0BB9E80011124080DA2
:1019D000191DF801859194910E94481AF8013496D6
:1019E000059114910115110509F464C081E060E0CE
:1019F0000E94A71910925E018EE591E0F801099509
:101A00008EE591E00E94831AE1E5E81B8E2F63E0EA
:101A10000E94BE198EE591E00E94551A4BC0F981D3
:101A2000F13009F047C086E49BE06BE47BE0A0DD89
:101A30006B2C7724842D90E00396861597051CF473
:101A40005DEF452E4B0CB41408F44B2CC42CDD2454
:101A5000C601880F991F8C0D9D1D880F991F880D39
:101A6000991D9D838C8300E010E07801EC0CFD1C37
:101A70002E143F04FCF0602F6F5F80E00E94BE19BF
:101A8000E614F70419F481E06EEF02C081E060E033
:101A90000E94A719EC81FD81859194910E94481ABA
:101AA0000F5F1F4FAC81BD811696BD83AC830430A0
:101AB0001105D9F60E947F198091C9029091CA023E
:101AC0008050944011F0AB2C04C0E1E0EB1508F01D
:101AD000A52C8091C9029091CA028050904211F0C9
:101AE000BA2C07C0A51418F0BB24B39402C0BA2CBA
:101AF000B3948091C9029091CA028038910511F483
:101B000080E01FC08091C9029091CA02049741F001
:101B10008091C9029091CA028050904809F02BCF61
:101B200086E0B89EF0011124E80DF91D32968591EA
:101B30009491009709F41FCFFC010995882309F4BB
:101B40001ACF0F900F900F900F900F90CF91DF91C1
:101B50001F910F91FF90EF90DF90CF90BF90AF90CB
:101B60009F908F907F906F905F904F903F902F90BD
:101B700008952F923F924F925F926F927F928F9231
:101B80009F92AF92BF92CF92DF92EF92FF920F930C
:101B90001F93DF93CF93CDB7DEB728970FB6F89496
:101BA000DEBF0FBECDBF6C01462E1A01298381E036
:101BB0008093CC02FF2499245524262F30E03B83C8
:101BC0002A83215030403D832C830E94C719B9DC01
:101BD000F60101900020E9F731978E2E8C18211420
:101BE000310489F082E060E80E94A719C1010E94D7
:101BF000711A86953AE2381B832F60E00E94BE1965
:101C0000C1010E94481A82E060E00E94A71982E4A4
:101C100060E00E94BE19682C77248A819B81861916
:101C2000970969E571E04AE050E00E94ED2B0E94BF
:101C3000551AFF2019F06EE57BE002C06BE47BE0F3
:101C40008981882319F089E69BE002C086E49BE045
:101C50008FDC81E060E00E94A71990E010E000E0D6
:101C6000EE2411C0EC0DFD1D80819E830E94601A40
:101C7000180F9E81123528F4F91609F4E02E9F5FA3
:101C800002C00F5F10E0E92FF0E06E167F0654F7F8
:101C9000802F6E2D52DDF914A0F410E010C0F60173
:101CA000E90DF11D80810E94601A282F812F90E09C
:101CB000820F911D8235910524F4120F9A94992078
:101CC00071F75F1438F5192DEE240EC01815F9F0D0
:101CD000F601E10FF11D80810E94601A080F0235A4
:101CE00010F41F5F02C0E39400E01F1578F30FC0EB
:101CF00010E0981451F0F601E90DF11D93948081E4
:101D00000E94601A180F1235A0F39A94EA9493E097
:101D10009E1570F3592CEE24BB24AA24B39480E0C2
:101D20006B2D0E94BE1900E010E01FC05F1441F44B
:101D3000EE2031F48FEF0E94BC19A12EEE24E39423
:101D4000EF81F88580810E94601A282F802F90E013
:101D5000820F911D823591058CF4020FEF81F88579
:101D600080810E942C1A53941F5F9601250D311D0E
:101D700038872F83F90180818823C1F6EE2039F45A
:101D8000581429F48FEF0E94BC19EE24E394F4E078
:101D9000BF1621F60E947F198091C9029091CA0254
:101DA000892B09F412CF8091C9029091CA020E9436
:101DB000C018282F833109F497C0843148F4813149
:101DC000E9F1823108F059C0863009F0A7C01BC084
:101DD000853149F0853108F482C0833219F18A32A5
:101DE00009F09CC08DC0FF2009F4BCC0FA948F2D6F
:101DF00090E0BC016F5F7F4F6C0D7D1D8C0D9D1DB4
:101E00000E948B2BE2CE2981222309F4ADC089EAFE
:101E100091E061E07DDD813009F4C0C0823008F4DA
:101E2000D4CEA2C08091CC028F5F0AB400FE02C063
:101E3000837001C081708093CC02C7CEEF2CEA186A
:101E400009F4C3CE1E2D00E0F601E10FF11D8081E3
:101E50000E94601A080F023510F41150A9F78A2D5C
:101E600090E0AC01410F511D2F2D30E0281B390BA4
:101E7000421753078CF1FE2CA8CE1F2D1A1900E033
:101E80000DC0F601E10FF11D80810E94601A080F5C
:101E9000023518F0F12E00E004C01F5F181588F31A
:101EA000F9CFF81451F0F601EF0DF11DF394808194
:101EB0000E94601A080F0235A0F32A2D30E0210F8E
:101EC000311D2615370514F0F82C7FCE8F2D90E0AC
:101ED000281739070CF079CEF12EFA0C76CEFF20B8
:101EE00009F473CEFA9471CE8F2D90E0EC81FD81D0
:101EF0008E179F070CF069CEF81408F066CE30C03C
:101F00000AB400FC06C08091C802882311F020E0CA
:101F100002C05BDC282F8AB58E7F8ABD203208F490
:101F200054CEF41419F00AB400FE04C08AB58160DE
:101F30008ABDFA940AB400FC0FC0942D07C0F601C4
:101F4000E90FF11D8291319680839150F916B8F313
:101F5000F601E80DF11D1182F601EF0DF11D208350
:101F6000F39433CE80E001C081E028960FB6F89458
:101F7000DEBF0FBECDBFCF91DF911F910F91FF90BC
:101F8000EF90DF90CF90BF90AF909F908F907F9019
:101F90006F905F904F903F902F900895FF2415CE43
:101FA0002F923F924F925F926F927F928F929F9269
:101FB000AF92BF92CF92DF92EF92FF920F931F9357
:101FC000DF93CF9300D000D000D0CDB7DEB783E051
:101FD0008093CC02BB24B394552453942EE5222E37
:101FE00021E0322E96E9492E0E94C719AADA89E12A
:101FF00060E00E94BE1982E060E80E94A71985E3B4
:102000009AE00E94481AAB2CAA948AE06A2D95DBCC
:1020100089E69BE06BE47BE0ABDA8B2C9924852D81
:1020200090E00396881599051CF48DEF582E5B0CF3
:10203000B51408F45B2C252D30E0C9010197AC01E3
:10204000440F551F480F591F440F551F440F551F6C
:102050004C5D5B4F5E834D8300E010E03A83298343
:102060009C838B83E980FA80E00EF11E5BE0E5162D
:10207000F1040CF08EC0602F6F5F80E00E94BE19EB
:10208000E814F90419F482E06EEF02C082E060E027
:102090000E94A7196B807C80600E711EED81FE810D
:1020A000608171818281938161157105810591053E
:1020B00009F463C00E94251DDC01CB016CE370E0D4
:1020C0000E94302C6C01643671051CF080E091E0B8
:1020D0002BC0CB016EE571E04AE050E00E94ED2B91
:1020E000F10101900020E9F7E056F14019F480E396
:1020F0000E942C1A8EE591E00E94551A8AE30E94F4
:102100002C1AC6016EE571E04AE050E00E94ED2B0A
:10211000F10101900020E9F7E056F14019F480E365
:102120000E942C1A8EE591E00E94551A80E20E94CE
:102130002C1AE814F90419F481E06EEF02C081E072
:1021400060E00E94A719F1012FE011922A95E9F7AA
:10215000B301660F771F660D771D660F771F660F39
:10216000771F685D7B4F8EE591E048E050E00E946C
:10217000AA2B8EE591E00E94551A0F5F1F4F4D81EB
:102180005E81445F5F4F5E834D830430110509F02B
:1021900069CF0E947F198091C9029091CA02805034
:1021A000944019F481E08B1508F0AB2C8091C902A2
:1021B0009091CA028050904231F4F9E0FA1518F07B
:1021C000BA2CB39401C0BA2C8091C9029091CA0272
:1021D00080389105D1F481E026960FB6F894DEBFE1
:1021E0000FBECDBFCF91DF911F910F91FF90EF9068
:1021F000DF90CF90BF90AF909F908F907F906F9027
:102200005F904F903F902F9008958091C9029091D8
:10221000CA028050904809F0E7CE84E892E061E07D
:1022200077DB823009F0E0CE8B2D90E00197BC0186
:10223000660F771F680F791F660F771F660F771F6E
:10224000685D7B4F8FEC92E048E050E00E94AA2B43
:10225000E3EEF2E0242D11922A95E9F783EE92E065
:1022600066E94DE752E021E084DCBECE3F924F921A
:102270005F926F927F928F929F92AF92BF92CF9216
:10228000DF92EF92FF920F931F93CF93DF93EC01B6
:10229000462E81E08093CC025B8868E0662E712C2C
:1022A0006C0E7D1EA42CBB2455E0AA0CBB1C5A95B9
:1022B000E1F742E1842E912C8A0C9B1CCC243AE25B
:1022C000332E8A89877090E08430910534F482300F
:1022D000910584F4019729F506C086309105A4F094
:1022E0000697F9F407C08EE591E063ED7AE00E946D
:1022F000652B17C08EE591E060E87BE00E94652BBE
:1023000081E691E0BE0109C08EE591E06CE77BE0DB
:102310000E94652B81E691E0B30148E050E00E9405
:10232000AA2B0E94C7190DD989E69BE06BE47BE0DC
:102330001FD982E060E80E94A7198EE591E00E9413
:10234000831A8695232D281B822F60E00E94BE19D8
:102350008EE591E00E94551A81E060E0F8D7DC2C10
:10236000EE24E39480E06E2D0E94BE19FF2415C078
:102370008E010D0D111DF80184890E94601A282F0D
:102380008F2D90E0820F911D8235910544F4F20E5D
:10239000F80184890E942C1AD394D51448F3F4E0F0
:1023A000EF16F9F6ACD78091C9029091CA02892B39
:1023B00071F08A898770853051F48AB5877F8ABD2C
:1023C0006A89687F64606A8BC4010E949C1F809147
:1023D000C9029091CA0224E08030920709F441C0FA
:1023E000E4E081309E0728F48038910509F069CF38
:1023F00057C0F0E280309F0729F08050904809F0E4
:1024000060CF02C010E049C08CE192E061E080DA68
:10241000823021F4842D0E946D2042C08330E9F483
:102420006A89862F8770863019F08230C9F506C018
:10243000687F6360C4010E949C1F43CF0E941C1DE3
:10244000998B888B8A89887F83608A8BC501BE01BE
:1024500044E150E00E94B61F23C0882309F431CF25
:102460001FC0CC2009F42DCF10E0FE01EC0DF11DB2
:1024700084890E94601A180F123508F022CFCA947E
:10248000A1F71FCFFE01EC0DF11D84890E94601A97
:10249000180F123508F015CFC394C51498F311CF57
:1024A000DF91CF911F910F91FF90EF90DF90CF9030
:1024B000BF90AF909F908F907F906F905F904F9064
:1024C0003F9008952F923F924F925F926F927F922A
:1024D0008F929F92AF92BF92CF92DF92EF92FF9234
:1024E0000F931F93DF93CF93CDB7DEB728970FB627
:1024F000F894DEBF0FBECDBF33243394BB24B39416
:1025000001C0B62C21E130E07724F999FECF32BD2D
:1025100021BDF89A80B5811173942F5F3F4F81E000
:102520002131380791F7772019F48AB5877F8ABD62
:1025300093E09093CC022BD704D889E160E01ED7BA
:1025400082E060E804D789E09AE0A2D76B2C6A9415
:10255000872D662DF2D886E89AE06BE47BE008D8F8
:10256000EB2DF0E0FA83E983832D90E003968E173C
:102570009F071CF4EDEF3E2E3B0CB31408F43B2CEC
:10258000222488249924EE24FF24232D30E03C8348
:102590002B83872D90E09E838D83CB80DC80CE0CB7
:1025A000DF1CED81FE81EC15FD050CF49AC06E2D4B
:1025B0006F5F80E0E3D630E0AA242FEF0DC0F999D9
:1025C000FECF822F90E08F5E9F4F92BD81BDF89A23
:1025D000A0B4A1103F5F2150832F90E08C159D0582
:1025E00074F30A2D10E075E0000F111F7A95E1F7E2
:1025F000C8016FEC72E04EE150E00E94E71F8FECE3
:1026000092E063E87AE00E94472B2C018091E1027E
:10261000877090E083309105F9F08430910534F4AF
:102620008130910561F0029779F413C085309105EE
:10263000F9F085309105BCF0069731F41EC082ECAC
:1026400099E023EE32E00CC080E090E018861F8213
:102650001AC08AEB99E013C082EB99E02FEC32E0CC
:1026600038872F8310C082EA99E0E7EDF2E009C0D5
:102670008AEA99E027ED32E0F3CF8AEC99E0EFECBB
:10268000F2E0F887EF834FD781E060E060D680E228
:10269000E3D629813A81C216D30629F481E06EEF90
:1026A00056D648012A2CEEE5F1E02FE011922A954A
:1026B000E9F78EE591E06F81788548E050E00E946F
:1026C000AA2B452819F481EE99E02DD78EE591E0EB
:1026D000ECD60894E11CF11C34E0E316F10409F097
:1026E0005CCF0DD68091C9029091CA02805094406F
:1026F00019F4F1E0FB1508F06B2C8091C902909160
:10270000CA028050904219F4671408F463948091CF
:10271000C9029091CA0280389105D1F480E02896D0
:102720000FB6F894DEBF0FBECDBFCF91DF911F91E2
:102730000F91FF90EF90DF90CF90BF90AF909F9060
:102740008F907F906F905F904F903F902F90089563
:102750008091C9029091CA02049741F08091C90208
:102760009091CA028050904809F0CBCE222009F403
:10277000C8CEC4016FEC72E044E150E00E94E71F54
:102780004091E20250E04B5E5F4FC4016FEC72E09B
:102790000E94E71F83E08093CC028FEC92E0622DD1
:1027A00065DDAFCE1F93CF93DF93F1D50E94A10AD1
:1027B00081E460E0E3D582E060E0C9D520919C042B
:1027C00030919D0484E690E0AC01249FC001259FD8
:1027D000900D349F900D112460E770E00E941C2C36
:1027E000CB01CEE5D1E0BE014AE050E00E94ED2BE6
:1027F000FE0101900020E9F7E156F14031F480E359
:102800002BD68EE229D6CE0107C080915E0124D658
:102810008EE222D6CE01019648D686E51DD683E00B
:102820008093CC020AB403FE05C089E69BE066E70C
:102830007BE004C089E69BE061E77BE00E94B80A88
:1028400088E160E09BD582E060E081D58AEE99E086
:102850001FD680E060E07BD5CEE5D1E01FE0FE0131
:10286000412F11924A95E9F7CE0169E471E048E001
:1028700050E00E94AA2BCE0146D6982F96958AE268
:10288000891B62E07BD5CE0110D6FE0111921A950C
:10289000E9F780915301882329F4CE0164E87BE0B5
:1028A0000E945A2B80915301813031F48EE591E0E2
:1028B0006CE87BE00E945A2B80915301823031F406
:1028C0008EE591E064E97BE00E945A2B8CE163E0A5
:1028D00055D582E060E03BD58EE591E0E6D5DF910D
:1028E000CF911F9108954FB7F8949C015D983EBD1C
:1028F0000DB407FEFDCF8EB5382F2EBD0DB407FEEB
:10290000FDCF8EB5282F5D9A4FBFC9010895906AFB
:10291000EACF80E090E0E7CF88EC92E8E4DF80ED5A
:1029200097E00197F1F781E89AECDDDF83E89AEC14
:10293000DADFEFDF80E090EBD6DF40984198429AF3
:102940008AB58D7F8ABD10920A01089582E0809336
:102950000A0180919C0490919D04823E910520F093
:1029600040984298419A03C040984198429A88E022
:1029700092E8B9DF88E392E8B6DF8AB582608ABD63
:1029800008959B01AC01283185E1380780E04807B4
:1029900080E0580760F460E678EA80E090E00E940A
:1029A000432CDA01C90101978068966C0AC06CEF6C
:1029B00072E485E090E00E94432CDA01C90101979E
:1029C000966C91CF88EE93E028EC30E0F9013197D6
:1029D000F1F70197D9F780EE90EC85DF87ED90E86D
:1029E00082DF8CEA92EC7FDF81E89AEC7CDF80E08A
:1029F00090EE79DF80E098EC76DF87EF94EC73DF80
:102A00008BDF80E197E20197F1F788E097E07FDFC5
:102A100080915301813019F488E29FE078DF809142
:102A20005301823019F487EA97E071DF88EA94E96C
:102A30005ADF60E875E280E090E0A3DF80E498E987
:102A400052DF6ADF66DF8AB18AB95B9A88E08093D9
:102A5000690082E08DBB089580910A01811181E0B7
:102A600008951F920F920FB60F9211240F931F9388
:102A70002F933F934F935F936F937F938F939F9386
:102A8000AF93BF93EF93FF9344DF97FF2AC08091EA
:102A90000A01813041F0813018F0823011F51DC0FB
:102AA00081E080930A0181E8A6D780E090EB1BDFEC
:102AB0008C0181E08ED7802F27D0882319F02CDF5E
:102AC00010920A0180910B01823058F080913B01F5
:102AD000882339F481E08FD704C0D1D190E0986B7E
:102AE00002DFFF91EF91BF91AF919F918F917F9105
:102AF0006F915F914F913F912F911F910F910F9087
:102B00000FBE0F901F901895EF92FF920F931F9397
:102B1000CF93DF93182FE0900E01F0900F0180917A
:102B20001101C82FD0E000913B0180910B01823050
:102B300009F45EC0833030F4882371F0813009F0ED
:102B40007EC13DC0843009F40DC1843008F4C2C098
:102B5000853009F074C171C1FE01E259FE4F108346
:102B60002196CE0104978B30910598F482599E4F9F
:102B70000E94072B882369F48091520183FF05C0CE
:102B800081E080930B0100E071C18FEF80930B0116
:102B90006DC1C130D10519F4EE24EA94FE2CC701B1
:102BA000612F0E942F2B7C01C431D10509F04EC149
:102BB000809181018A5E8093100183E03AC1E02F09
:102BC000F0E0E254FB4F10830F5F033109F03EC188
:102BD00082E080930B0110923C0110923D01109213
:102BE0003F0110923E0180E0C0E0D0E00FE02FC135
:102BF000FE01E259FE4F10832196C130D10519F430
:102C0000EE24EA94FE2CC701612F0E942F2B7C0139
:102C1000C431D10531F483E080930B018CEA8093B9
:102C20001001CE0183709070892B09F00FC1789448
:102C300080913C0160913D0190E070E062547B4FD7
:102C400082599E4F40E028E00E94EF29282F8430CF
:102C500030F08FEF80930B0188EC90E02BC08091D7
:102C60003C018C5F80933C0180913D018D5F80939E
:102C70003D0180913E0190913F01820F911D909303
:102C80003F0180933E01C431D10508F4DFC080913B
:102C900081018823A1F0809181018A5E80931001D7
:102CA00080918101873908F4D1C08FEF80930B01A7
:102CB00080EF90E090933F0180933E0136C08FEF0C
:102CC00080930B0187E990E090933F0180933E0150
:102CD0009FD1BCC0FE01E259FE4F10832196C7016F
:102CE000612F0E942F2B7C0120911001822F90E0F8
:102CF000C817D90709F0AAC0273120F0FE01E4590E
:102D0000FE4F1082002399F486E990E090933F01F2
:102D100080933E01E114F10429F485E080930B01D6
:102D2000789476D18FEF80930B0181E090C084E09E
:102D300080930B018091810190E0880F991F69E0D9
:102D400070E00E94302C6F5F062F000F060F265197
:102D50002093100110923D0110923C01109240010D
:102D600080E03AC080913D01E82FF0E0E254FB4F53
:102D700010838F5F80933D012196C330D10509F008
:102D80004CC080913D01801711F029E009C080916D
:102D90003C019091400120911001281B220F291B1A
:102DA000789480913C0160913D014091400190E018
:102DB00070E065547B4F8E579E4F0E94EF29282F5D
:102DC000843068F08FEF80930B0189EC90E0909352
:102DD0003F0180933E0181E0C0E0D0E038C08091A7
:102DE0003C018C5F80933C0190913C0180914001BB
:102DF000890F80933C0180913E0190913F01820FA9
:102E0000911D90933F0180933E018091400191E09C
:102E1000892780934001C0E0D0E080913D01801778
:102E2000A8F080EA90E090933F0180933E01F0D0BB
:102E30008FEF80930B0180E007C0000007C0109265
:102E40000B0181E0C0E0D0E000E001C080E0F09242
:102E50000F01E0920E0100933B01C0931101DF913D
:102E6000CF911F910F91FF90EF900895C0E0D0E0B7
:102E700096CE52DD85E080936D0181E0BCC59091D6
:102E80002D0280910C01833009F455C0843030F458
:102E9000813089F1823008F03CC00AC0853009F4E5
:102EA0006AC0853008F451C0863009F090C079C0FE
:102EB00080915201E0910D0183FF11C0E33148F48C
:102EC000EF5FE0930D01E150F0E0E25DF64F849199
:102ED000089510920D0181E080930C010CC082E0F6
:102EE00080930C01EF5FE0930D01E150F0E0E65DAF
:102EF000F64F8491089520910D012F3028F4E22F90
:102F0000F0E0E254FB4F2DC010920D0182E080935F
:102F10000C01E0910D01E43048F4EF5FE0930D0106
:102F2000E150F0E0E65DF64F8491089510920D01B6
:102F300083E080930C0120910D01243118F4E22FDD
:102F4000F0E00DC084E080930C0120910D01E22F90
:102F5000F0E0892F90E04496E817F90738F4E65E30
:102F6000FD4F80812F5F20930D01089585E08093B0
:102F70000C0110920D0190910D01923028F4E92F6F
:102F8000F0E0EC53FD4F17C010920D0180915201FB
:102F900083FD04C087E080930C0117C086E0809316
:102FA0000C0190910D0180913B01981748F4E92F95
:102FB000F0E0E353FB4F80819F5F90930D010895F4
:102FC00087E080930C0110923B018AEA08951092E9
:102FD0000D0110920C014DDF8AB58D7F8ABD80E016
:102FE00008953ADD882329F0789436DD8823E9F7BF
:102FF000F89410920C01AACC2FDD882319F081E0FF
:1030000090E0089586DC892F99278170907008954B
:10301000CF93DF938EE691E064E479E00E94472B42
:10302000EC018091520182FD02C020E00AC08EE6D0
:1030300091E061E479E00E94472B20E0892B09F4BC
:1030400021E0CD2B71F0222361F48EE691E069E45A
:1030500071E048E050E00E94922B892B11F080E053
:103060000FC04091810150E04B5E5F4F89E793E0D4
:103070006EE671E00E947B2B8AB580688ABD81E094
:10308000DF91CF910895EF92FF920F931F93CF930B
:10309000DF937C0180E09DD40FEF1FEFC0E0D0E014
:1030A00009C0FE01E65EFD4FC80160810E942F2B22
:1030B0008C012196F701838990E04496C817D907BF
:1030C00080F38091520183FF05C0C7016EEB74E06D
:1030D0000E946A251093C5020093C40282DF80918A
:1030E000520183FF0AC0C70144966DEC74E0F701FA
:1030F00043890E94D22280933B0180E07CD480E00F
:10310000DF91CF911F910F91FF90EF90089582E092
:103110008093CC021092CA021092C9021092C70288
:103120001092C602E8E6F0E0808184608083089512
:103130009FB7F894E8E6F0E0808184608083509A3D
:10314000519A58985998589A599A50988AB18C7FA0
:103150008AB99FBF08951F920F920FB60F92112444
:103160008F93EF93FF93E8E6F0E080818B7F80837D
:10317000FF91EF918F910F900FBE0F901F901895B8
:103180009C018AB58E7F8ABD4FB7F8948FE18093FA
:10319000C8028091C6029091C7028217930749F432
:1031A0008091CB028F5F8093CB028AB581608ABD0C
:1031B00002C01092CB023093C7022093C6024FBFC9
:1031C000EFE0E15021F03695279520FFFACF80916E
:1031D000CC02833059F41092CB02F0E0EE0FFF1FC7
:1031E000EE0FFF1FE156F44F84910895F0E0823016
:1031F00051F41092CB02EE0FFF1FEE0FFF1FE256AD
:10320000F44F849108959FB7F894EE0FFF1FEE0FCF
:10321000FF1FE456F44F259134912115310519F41F
:103220009FBF80E008958091CB02F901E80FF11D66
:10323000E491EE2331F480E0F8CF8E2F90E00C94EF
:10324000652C8093CB029FBF8091CC028130A9F383
:103250008E2F08951F9319B11370133019F480E065
:1032600090E043C084E0B5D38091520180FF06C056
:103270000AB404FE03C08AB580628ABD20E030E053
:10328000412F10FF0FC05C985098519A00009FB7D3
:10329000F8945C9A1EBC0DB407FEFDCF51988EB514
:1032A000282F9FBF41FF0FC05C98509A5198000093
:1032B0009FB7F8945C9A1EBC0DB407FEFDCF5098E2
:1032C0008EB5382F9FBF1092680083E08BBB309380
:1032D00048012093470184E08ED38091470190916B
:1032E000480110924801109247011F910895B2DFE2
:1032F000009721F09093CA028093C9020895CF935A
:10330000DF93C0E2DEE410C00BB400FE0AC01092EE
:10331000CA021092C9028BB58E7FEAE4F0E0818385
:1033200013C0CE010197F1F795DF892B69F307C030
:103330000BB400FC09C0CE010197F1F702C0C0E256
:10334000DEE4D5DF892BA1F7DF91CF91089580933B
:1033500012016093130108952FB7F8949FEE9BB963
:103360008EBD5A9861115A9A0DB407FEFDCF5C9A32
:103370002FBF089560E0F0CF61E0EECF1F93162FCE
:103380008058F8DF812F805CF5DF1F910895CF937F
:10339000DF93C8EFD1E080E0EFDF2197E1F7DF9125
:1033A000CF9108951092130181E080931201449807
:1033B00080ED97E0FC013197F1F7449A0197F1F71E
:1033C00080E29EE40197F1F781E2D4DF8091510120
:1033D000885D8068CFDF86E0CDDF83E1CBDF80E2F0
:1033E000C9DF8CE0C7DFD3CF982F8B3718F18F3D23
:1033F000D1F0803E38F4863D69F18C3D61F0843C2B
:10340000A1F407C0863F59F08C3F59F0843E69F41F
:1034100004C09BE70FC09DE70DC09EE70BC09FE770
:1034200009C090E807C091E805C0923818F080E024
:1034300090E00895905283E0989FF00111248091CC
:103440001201E80FF11DEE0FFF1FE654F94F8591B1
:10345000949108959CE7EECF0F931F93CF93DF9342
:10346000C3DFEC01009761F08E012196F801049111
:10347000802F8E7F9091130189277EDF00FFF4CF8C
:103480008091130179DFDF91CF911F910F91089502
:10349000CF93DF93EC0101C0DFDFFE012196849121
:1034A0008823D1F7DF91CF910895CF93DF93EC017B
:1034B00001C0D2DF89918823E1F7DF91CF91089590
:1034C00093DF009711F440E009C09C01F9012F5FE0
:1034D0003F4FE491422F481BE0FFF8CF842F8F5FCE
:1034E00008951F93CF93DF93EC0110E002C0E8DF53
:1034F000180FFE01219684918823C9F7812FDF914F
:10350000CF911F9108951F93CF93DF93EC0110E0AB
:1035100002C0D6DF180F89918823D9F7812FDF9158
:10352000CF911F910895FF920F931F93CF93DF9335
:10353000EC018C01FC01F49004C02196FE01849101
:103540001BDF9E01201B2F15C0F3DF91CF911F9130
:103550000F91FF9008951092CD0282EA809380002F
:1035600082E080938100109289001092880010926E
:103570008B0010928A00089510921C0110921E0177
:103580001092230410921D010895FF920F931F9330
:10359000CF93DF938BB58D7F8BBD90E8F92E01E043
:1035A000F999FECFF999FECF802F90E08F5E9F4F63
:1035B00092BD81BDF89A80B5882319F1C82FD0E05B
:1035C00085E0CC0FDD1F8A95E1F7CE016FE171E058
:1035D00044E150E0FCD410913101812F8770863096
:1035E00081F48FE191E064E171E048E050E00E94F5
:1035F000922B892B31F4187F1360CE014296612FF4
:103600009BD4FA940E5FFF2059F6DF91CF911F9162
:103610000F91FF9008950F931F93CF93DF930AB4F8
:1036200007FEE8C080918B0386958695869583700A
:1036300090E08130910509F444C083309105B1F0E8
:10364000892B09F0C4C081E893E053D30BB401FC8B
:103650000BC084E191E061E873E048E050E00E9433
:10366000AA2B8BB582608BBD90DFB1C020912A025E
:1036700030912B028091890390918A032817390792
:1036800009F0A5C08AE192E061E873E048E050E00B
:103690000E94922B892B09F09AC000911C0110E026
:1036A00045E0000F111F4A95E1F70E5E1F4FC8015C
:1036B00024D4682F687F6260C8013ED4109223042E
:1036C00086C001E110E0F999FECF12BD01BDF89A64
:1036D00080B5882329F1C82FD0E035E0CC0FDD1F5D
:1036E0003A95E1F7CE01429608D48C5F877082301C
:1036F000B8F4CE016FE171E044E150E068D420916C
:10370000890330918A0380912F019091300128170D
:10371000390731F490918C0380913201981769F147
:103720000F5F1F4F81E00131180769F654C0802FE9
:1037300090E0412F50E025E0880F991F2A95E1F78E
:1037400069E773E013D4802F612F01D58AB58062B9
:103750008ABD8AB588608ABD8BB581608BBD80913A
:10376000540180FF03C080E28093CD028091540118
:1037700081FF03C088E08093CE0289E793E063E88D
:103780007AE00E94472B892B11F182E292E069E4F2
:1037900071E048E050E00E94AA2B8AE192E061E8E3
:1037A00073E048E050E00E94AA2B10922D02809115
:1037B0002C02886180932C028091890390918A0366
:1037C00090932B0280932A0282E0809323048AB58F
:1037D0008F778ABD0FC080918B03887F856080932F
:1037E0008B0310918C031B5E812F4BD4082F8823F1
:1037F00071F39DCFDF91CF911F910F9108950F939A
:103800001F93CF93DF9328D9882309F09DC080911F
:103810002304813009F46CC0813038F0823009F41F
:1038200089C0833009F090C03BC01FEFF999FECFEB
:1038300080911E018F5F80931E01F999FECF90E069
:103840008F5E9F4F92BD81BDF89A00B5002319F19C
:10385000C02FD0E075E0CC0FDD1F7A95E1F7CE01E7
:1038600042964BD387708330B1F4CE016AE172E0A7
:103870004AEA50E0ACD300931C018091560190E0DD
:1038800063E0880F991F6A95E1F780931D0181E03D
:103890008093230459C0112309F456C01150C6CF98
:1038A000109223048AE192E060E070E04AEA50E07E
:1038B0000E94842B82E292E069E471E048E050E0EB
:1038C0000E94AA2B8AE192E06BE17CE048E050E0A4
:1038D0000E946C2B80912C02877E80932C02809119
:1038E0002C02887F836080932C0210922D0229C0C5
:1038F00080911D01882351F0815080931D018F5FBD
:1039000090E087709070892BF9F41BC000911C0126
:1039100010E055E0000F111F5A95E1F70E5E1F4FA2
:10392000C801EBD2682F687F6660C80105D310928A
:1039300023040AC080911E01815080931E011092C1
:1039400023048AE192E09FDBDF91CF911F910F91D9
:103950000895FF920F931F938091E102877E886004
:103960008093E10287ED92E069E471E048E050E085
:103970000E94AA2BE3EEF2E001900020E9F7E45E5A
:10398000F240E093E20258D09093E0028093DF028D
:103990000091E2020B5EFFB6F894802F72D3182FCD
:1039A000882319F4FFBE80E010C090E0402F50E063
:1039B000E5E0880F991FEA95E1F76FEC72E0D6D247
:1039C000812F602FC4D3FFBE81E01F910F91FF9024
:1039D000089590913401982B909334019FB7F894F7
:1039E000E1E6F0E080E88083108287E08093B10018
:1039F0001DBC9FBF089508958EE18093370123E099
:103A0000209336018091570190E090933A01809382
:103A1000390116BC10926E0025BD109285001092DF
:103A20008400109238018FE1809335011092B2002A
:103A300081E080937000089580914301909144014A
:103A4000A0914501B0914601089520914301309124
:103A500044014091450150914601261B370B480B0C
:103A6000590BCA01B9012CE330E040E050E00E945C
:103A7000432CCA01B90108951F920F920FB60F92FD
:103A800011242F933F934F935F936F937F938F9363
:103A90009F93AF93BF93EF93FF9382E09ADF809160
:103AA000C802882329F41092C7021092C60205C0EA
:103AB0008091C80281508093C8020AB404FE78C085
:103AC0004091350140FF20C02091CD022223E1F03A
:103AD00084E59CE6A4E1BDEA022E04C0B695A79554
:103AE000979587950A94D2F780FF07C088ED90E0FC
:103AF000909389008093880004C0109289001092EE
:103B0000880021502093CD020AB405FE17C0809191
:103B10008A0090918B00809621E0803E920738F4D5
:103B200090938B0080938A00109238011CC08FEF15
:103B300091E090938B0080938A0015C020918A00B9
:103B400030918B0080918A0090918B00409738F0E3
:103B50002051304030938B0020938A0004C0109293
:103B60008B0010928A000AB401FC18C04F3011F08B
:103B70004423A1F42091CE02222381F088EA90E030
:103B8000022E02C0959587950A94E2F780FF02C045
:103B9000409A01C0409821502093CE028091380174
:103BA000815080933801882319F48AB58F7D8ABDAE
:103BB00080913301882309F08BC080913B018823D9
:103BC00009F086C081E080933301789424DD8091F0
:103BD00035018F3009F413DE30913501343101F5B0
:103BE00080915701882309F46EC08091390190912A
:103BF0003A01009779F480912304882309F063C087
:103C000083E080932304809157012CE3829FC001BD
:103C1000112401C0019790933A018093390153C058
:103C2000332309F050C08091430190914401A09149
:103C30004501B09146010196A11DB11D809343013C
:103C400090934401A0934501B09346018FE1809386
:103C500035010AB404FC1AC0499905C08091680076
:103C6000846080936800F6DA8038910521F48091B1
:103C70003601815001C083E0809336018091360186
:103C8000882321F58AB580618ABD20C0E3DA8034BB
:103C9000910521F480913601815001C083E0809329
:103CA000360180913601882309F4000080913701A4
:103CB000882329F48EE180933701D2D007C0815048
:103CC0008093370103C03150309335011092330196
:103CD000FF91EF91BF91AF919F918F917F916F91E4
:103CE0005F914F913F912F910F900FBE0F901F90BA
:103CF0001895CF92DF92FF920F931F93CF93DF938C
:103D00006C0100E010E0F02EE801CC0FDD1FC00FC9
:103D1000D11FCC0FDD1FCC0FDD1FBE01685D7B4FB7
:103D2000C60148E050E00E94922B892B59F4FE0115
:103D3000EC5DFB4F20813181428153818AE008177D
:103D400041F41AC00F5F1F4F0A301105E1F62AE057
:103D500014C08091430190914401A0914501B0911C
:103D60004601821B930BA40BB50B89559240A040D2
:103D7000B04010F4202F25C02F2D8AB580628ABD57
:103D80008091550180FF03C084E08093CD02809133
:103D9000550181FF16C086E08093CE0212C02A3002
:103DA00070F4239FC0011124DC01AC5DBB4FFC010A
:103DB000E85EFB4F8CE001900D928150E1F72150BD
:103DC00001C03CE0222359F788E294E0B60148E0C4
:103DD00050E00E94AA2B8091430190914401A09150
:103DE0004501B09146018093240490932504A0934B
:103DF0002604B0932704DF91CF911F910F91FF907C
:103E0000DF90CF9008950F931F93CF93DF93E4E259
:103E1000F4E088E7DF011D928A95E9F78F01C0E0A1
:103E2000D0E0F8011082118212821382CE01880F35
:103E3000991F8C0F9D1F880F991F880F991F885DF0
:103E40009B4F62E07AE00E94652B2196045F1F4F32
:103E5000CA30D10531F7DF91CF911F910F910895AD
:103E600080E880BF3D9AE4E6F0E080818E7F808329
:103E700010929D0410929C0487E480937C008DED49
:103E800080937A0008951F920F920FB60F9211241B
:103E90008F939F933D988091780090917900813520
:103EA000910540F0809178009091790090939D0465
:103EB00080939C0480917A008F7780937A00809120
:103EC00064008160809364009F918F910F900FBE7A
:103ED0000F901F9018958EBD0DB407FEFDCF08956D
:103EE0005F9885E0F8DF80E0F6DF5F9A0EB400FCB3
:103EF000F7CF82E08A95F1F70895FF920F931F9311
:103F00008C01FFB6F894ECDF5F9883E0E4DF812F4B
:103F1000E2DF802FE0DF80E0DEDF5F9AFFBE8EB55C
:103F20001F910F91FF9008955F9886E0D4DF5F9A0C
:103F300082E08A95F1F70895EF92FF920F931F9315
:103F40008C01F62EEFB6F894CBDFEEDF5F9882E0BF
:103F5000C2DF812FC0DF802FBEDF8F2DBCDF5F9AD5
:103F6000EFBE1F910F91FF90EF900895DF92EF92B7
:103F7000FF920F931F93CF93DF93EC017B018A0194
:103F8000DFB6F894ADDFD0DF5F9882E0A4DF8D2F3D
:103F9000A2DF8C2FA0DFF70181917F019CDF015010
:103FA00010402196CE018F719070892B19F0011568
:103FB000110589F75F9A0115110521F7DFBEDF9121
:103FC000CF911F910F91FF90EF90DF900895DF92B6
:103FD000EF92FF920F931F93CF93DF938C017B019E
:103FE000EA01DFB6F8947CDF5F9883E074DF812F0D
:103FF00072DF802F70DF07C080E06DDF8EB5F701C4
:1040000081937F0121972097B9F75F9ADFBEC7019F
:10401000DF91CF911F910F91FF90EF90DF90089566
:10402000282F662311F480E00895862F90E00197F1
:1040300060E270E00E94302C6F5F1FC0922F97707B
:10404000822F869586958695A82FB0E0FD01E256D1
:10405000FB4F8081E92FF0E0442329F0E25EF34F2B
:104060009491982B05C0E25EF34F9491909598231C
:10407000A256BB4F9C932F5F61506623F9F681E0F7
:10408000089590E0019760E270E00E94302C6F5F2D
:1040900040E031E0E32FE695E695E695F0E0E25664
:1040A000FB4F808190E0232F277002C09595879564
:1040B0002A95E2F780FD07C04F5F461729F4832F4A
:1040C000841B8F5F089540E03F3F11F03F5FE2CFD8
:1040D0008AB580648ABD80E008950F931F93182FDE
:1040E00021E130E0F999FECFF999FECF32BD21BD33
:1040F000F89A80B5811701F50FB7F894F999FECFBA
:10410000F999FECF1FBA32BD21BD10BC0FB6F8948D
:10411000FA9AF99A0FBE812F90E025E0880F991F37
:104120002A95E1F74396E9DE682F6C5E812F40E027
:1041300077DF0FBF81E008C081E02031380719F038
:104140002F5F3F4FCFCF80E01F910F910895782FC1
:1041500020E031E001C09A01F999FECFA901415058
:104160005040CA018F5E9F4F92BD81BDF89A80B5C5
:10417000882389F381E02030380711F480E0089526
:10418000F999FECFF999FECF1FBA2F5E3F4F32BD8E
:1041900021BD70BD0FB6F894FA9AF99A0FBE872F19
:1041A00041E03EDF81E008951F93CF93DF9380E2EB
:1041B000EEE9F4E0DF011D928A95E9F781E0809352
:1041C0009E04C1E1D0E0F999FECFF999FECFD2BDAE
:1041D000C1BDF89A10B5112379F0812F90E035E038
:1041E000880F991F3A95E1F7439687DE682F6C5E3A
:1041F00019F0812F41E014DF2196B1E0C131DB07D6
:1042000011F7DF91CF911F9108951F931FB7F89475
:1042100020E030E0822FF999FECFF999FECF1FBA46
:1042200090E08F5E9F4F92BD81BD10BC0FB6F89499
:10423000FA9AF99A0FBE2F5F3F4F81E0203038077E
:1042400049F7B2DF1FBF1F91089580E008959FD8FE
:1042500082E060E87CD88FE060E090D888E59CE060
:1042600017D90E94A10A81E060E071D880E061E086
:1042700085D887E89CE00CD980E062E07FD881E8AF
:104280009CE006D980E063E079D884E79CE000D91F
:1042900080E064E073D888E69CE0FAD886E49BE08E
:1042A00060E070E00E94B80A2AD88091C90290911B
:1042B000CA028050924019F4E9980E94A614809195
:1042C000C9029091CA028050944031F40E948C142B
:1042D0000E94891482E08DBB8091C9029091CA022C
:1042E0008050984029F4E9980E94A6144198429A77
:1042F0008091C9029091CA02809781F481E464E0C0
:104300003DD880919C0490919D046EE571E04AE057
:1043100050E00E94ED2BC9D80E947F198091C902FC
:104320009091CA028050904809F091CF80E00895A2
:1043300087E19BE060E00E94680B882369F0F894B5
:1043400028E088E190E00FB6F894A895809360008B
:104350000FBE20936000FFCF1AD882E060E80E9471
:10436000A71984E160E00AD880E59CE091D880E05C
:1043700061E004D88BE99CE08BD881E060E00E948A
:10438000A71980E269D88AEE99E082D880E264D8E1
:1043900087E499E07DD880E062E00E94BE1982E067
:1043A00060E80E94A71988E99CE072D881E060E08B
:1043B0000E94A71980E250D880E699E069D882E08F
:1043C00060E80E94A71980E063E00E94BE1985E9B9
:1043D0009CE05ED882E060E00E94A71980E23CD8B1
:1043E0008BE499E055D880E237D887E599E050D83A
:1043F00086E49BE060E070E00E94B80A0E947F19AA
:104400008091C9029091CA028050904809F0A4CFCF
:1044100080E00895EF92FF920F931F93CF93DF9365
:104420000E94C71985E060E00E94BE1982E060E842
:104430000E94A7198FE99CE02BD883E061E00E94DD
:10444000BE1901E0C0E0D0E081E0E82EF12CCE0101
:104450006FE370E00E941C2C892BD9F4209749F05F
:1044600080E00E94BC198FEF0E94BC198FEF0E9460
:10447000BC19102F1F5F83E0602F0E94BE198FEFC1
:104480000E94BC198FEF0E94BC1980E00E94BC19E9
:10449000012FCE0168E070E00E94302CDC01CB01DE
:1044A000970102C0220F331FAA95E2F782569B4F55
:1044B000FC01808190E0822393238217930711F4FB
:1044C0008CE901C080E80E94BC192196F1E0C0305F
:1044D000DF0709F0BCCF80E00E94BC198FEF0E947B
:1044E000BC198FEF0E94BC1982E06EE70E94A719E9
:1044F00080E065E00E94BE1986E49BE00E94481AB5
:104500000E947F1980E0DF91CF911F910F91FF9062
:10451000EF9008958295807F682BE2EEFCE0E60F35
:10452000F11DE4918E2F08958295807F682B82EE95
:104530009CE0FC01E60FF11DE4914295407FE42BE5
:104540008E0F911DFC0184910895E2EEFDE0E80FCD
:10455000F11DE4918E2F0895E2EFFDE0E80FF11DCB
:10456000E4918E2F08951F93182F613071F0862FDC
:10457000ECDF9FE0981B892FEFDF1295107F182B3F
:10458000E12FF0E0EE51F34F84911F910895982FA1
:104590009295907F982BE2EEFCE0E90FF11DE491FB
:1045A0008E2F08952F923F924F925F926F927F923B
:1045B0008F929F92AF92BF92CF92DF92EF92FF9233
:1045C0000F931F93DF93CF93CDB7DEB728970FB626
:1045D000F894DEBF0FBECDBF3C017B836A83842E7F
:1045E0001B01198225C1D3011D91B887AF83B98101
:1045F000BB2349F4EFE0DE2ED122E12EE2947FE0EE
:10460000E722EBEF0AC0D12ED2946FE0D622D3017D
:104610001196EC90BFE0EB22ECEF8E0E8FE06D2D4B
:1046200079DFF82E87E06E2D75DF182F6E2D6D2542
:1046300089E070DFA82EA29450EFA5221F25A12AA1
:1046400085E06D2D67DFC82E83E06E2D63DF182FA8
:1046500088E06D2D5FDF082F8CE06E2D5BDF082773
:104660000295007F1C25012B8AE06E2D53DF182F49
:104670008D2D67E04FDFE8268CE06E2D4BDF982E06
:10468000929440EF94221F25912A4F8058840894D9
:10469000411C511CBB24B394AF81B8858C91B98166
:1046A000BB2339F4282F2F70982F92959F703201D9
:1046B00007C0282F22952F703201F20190819F7040
:1046C0003FE0F32EFA20F22687E06F2D9E8322DF53
:1046D0001A2D12951F7018279E811927812F67E0C8
:1046E00019DFE82E8F2D69E015DFD82E812F69E0C4
:1046F00011DFA82E8F2D63E00DDF902F907FA8266D
:10470000A29480EFA822A9260F70DE240D25A02AEE
:104710008F2D6CE0FFDEE82E812F63E0FBDEC82EDC
:10472000812F6CE0F7DED82E8F2D6AE0F3DE992D15
:10473000907F082F0D250295007F0927FFE09F221B
:10474000CE249C240929812F6AE0E4DE9D2C9294DA
:1047500010EF9122E8269E28B3940894411C511C26
:104760004F8158854F5F5F4F58874F8354E0B51690
:1047700009F092CFD3011C91B981BB2319F4612FA9
:104780006F7006C0612F62956F700894611C711C78
:10479000E981F1E0EF27E9831A2D1F701627812F99
:1047A00067E0B8DEB82E812F69E0B4DEE82E812FF5
:1047B0006CE0B0DEC82E812F63E0ACDE582EDD2425
:1047C000812F6AE0A7DE202F30E02F703070FF24A9
:1047D0002E253F25B4E0220F331FBA95E1F7A294AE
:1047E000AFE0AA22AB24A22AD101AC92292D30E05D
:1047F0002F7030702C253D25F4E0220F331FFA95E1
:10480000E1F702950F700525022B11960C93119775
:104810009294EFE09E22982674E0CC0CDD1C7A95F1
:10482000E1F79C2812969C92E3E0F0E02E0E3F1EEA
:10483000522CFA815F1A24E0281508F4D4CE882D72
:1048400090E04981840F911D892B09F429C18820AA
:10485000E1F0D3011D91B887AF83482D4150B98154
:10486000BB2341F46FE0D62ED122E12EE2945FE02B
:10487000E52209C0D12ED2943FE0D322D301119674
:10488000EC90BFE0EB22B42E0BC0F301D190F8877F
:10489000EF83D2942FE0D222BB24BA94EE24198263
:1048A0008FE06D2D37DEF82E87E06E2D33DE182F6A
:1048B0006E2D6D2589E02EDE982E929490EF992230
:1048C0001F25912A85E06D2D25DEC82E83E06E2DF3
:1048D00021DE182F88E06D2D1DDEA82E8CE06E2DB8
:1048E00019DEA826A29480EFA8221C25A12A8AE01E
:1048F0006E2D10DE182F8D2D67E00CDEE8268CE083
:104900006E2D08DE882E829400EF80221F25812ADA
:1049100077247394BB20C9F0EF81F88521914B2D4A
:1049200041505981552341F4322F3F70022F029597
:104930000F70F887EF8307C0322F32953F70F887EA
:10494000EF8300810F70B42E0FC08981882319F482
:1049500030E000E009C0AF81B8853D91B887AF83F2
:1049600032953F7000E01982BFE0FB2EF920F3265C
:1049700087E06F2DCFDD192D12951F701827102796
:10498000812F67E0C7DDE82E8F2D69E0C3DDD82ECB
:10499000812F69E0BFDD982E8F2D63E0BBDD9A2D5E
:1049A000907F98269294A0EF9A229926BFE0AB229E
:1049B000DE24AD249A288F2D6CE0ACDDE82E812F0B
:1049C00063E0A8DDC82E812F6CE0A4DDD82E8F2DEA
:1049D0006AE0A0DD982D907FA82EAD24A294F0EF80
:1049E000AF22A926EFE08E22CE248C24A828812F86
:1049F0006AE090DD8D2C8294E0EF8E22E8268E28EE
:104A00007394F4E07F1609F085CF7FE0D72ED9208C
:104A10008D2D67E07FDDB82E8D2D69E07BDD182FB1
:104A20008D2D6CE077DDE82E8D2D63E073DDC82ED3
:104A3000FF248D2D6AE06EDD2A2D30E02F7030705E
:104A4000412F50E02427352764E0220F331F6A9559
:104A5000E1F792945FE095229B24922AF1019192D2
:104A6000282D30E02F7030702E253F2544E0220F96
:104A7000331F4A95E1F7A2943FE0A322AC24A22A77
:104A8000D1011196AC9282949FE08922882684E01D
:104A9000EE0CFF1C8A95E1F78E288182B3E05B0E55
:104AA000852D28960FB6F894DEBF0FBECDBFCF91EF
:104AB000DF911F910F91FF90EF90DF90CF90BF900B
:104AC000AF909F908F907F906F905F904F903F90AE
:104AD0002F9008952F923F924F925F926F927F9204
:104AE0008F929F92AF92BF92CF92DF92EF92FF92FE
:104AF0000F931F93DF93CF9300D00F92CDB7DEB704
:104B00002B011C018824D101ED913D01FE2EFFE017
:104B1000FF22CE2EC294BFE0CB228FE06F2DFADCB5
:104B2000D82E87E06C2DF6DC182F6C2D6F2589E0D0
:104B3000F1DCA82EA294A0EFAA221D25A12A85E0CF
:104B40006F2DE8DCE82E83E06C2DE4DC182F88E084
:104B50006F2DE0DC082F8CE06C2DDCDC0827029543
:104B6000007F1E25012B8AE06C2DD4DC182F8F2DA1
:104B700067E0D0DCC8268CE06C2DCCDC982E9294BB
:104B8000F0EF9F221D25912A44E050E0240E351EAF
:104B9000D3011D913D01F12EFA24BFE0FB2287E0F5
:104BA0006F2DB8DC12951F701827A294EFE0AE228B
:104BB0001A25812F67E0AEDCE82E8F2D69E0AADC94
:104BC000D82E812F69E0A6DCA82E8F2D63E0A2DC11
:104BD000902F907FA826A29470EFA722A9260F708D
:104BE000DE240D25A02A8F2D6CE094DCE82E812F89
:104BF00063E090DCC82E812F6CE08CDCD82E8F2DEA
:104C00006AE088DC992D907F082F0D250295007FA2
:104C10000927EFE09E22CE249C240929812F6AE0F7
:104C200079DC9D2C929460EF9622E8269E286214EF
:104C3000730409F0ADCF5FE0D52EDA208D2D67E04B
:104C400069DCB82E8D2D69E065DC182F8D2D6CE0A8
:104C500061DCE82E8D2D63E05DDCC82EFF248D2DF8
:104C60006AE058DC202F30E02F703070412F50E088
:104C70002427352744E0220F331F4A95E1F7A294F9
:104C80003FE0A322AB24A22AD201AC92292D30E02E
:104C90002F7030702E253F2594E0220F331F9A95F8
:104CA000E1F702950F700C25022B11960C931197CA
:104CB00092941FE091229826F4E0EE0CFF1CFA95E6
:104CC000E1F79E2812969C928394B5E08B1631F002
:104CD000E3E0F0E04E0E5F1E130115CF0F900F9032
:104CE0000F90CF91DF911F910F91FF90EF90DF9088
:104CF000CF90BF90AF909F908F907F906F905F907C
:104D00004F903F902F9008953F924F925F926F92F5
:104D10007F928F929F92AF92BF92CF92DF92EF924B
:104D2000FF920F931F93CF93DF936C013B01542E9F
:104D3000E901402EEE243324339449010894811C68
:104D4000911C22E0A22EB12CAC0EBD1EE41410F07A
:104D5000FF2410C0F6011081552021F49FE0F92EA8
:104D6000F12207C0F12EF2948FE0F8220894C11CC2
:104D7000D11C53240881802F8F7062E0CBDB182F69
:104D8000802F82958F7064E0C5DB8F258295807FB0
:104D90001F25812B8883F4010081802F8F7068E0AC
:104DA000B9DB182F802F82958F7063E0B3DB8F25DE
:104DB0008295807F1F25812BF4018083F50110816E
:104DC000812F8F7066E0A6DB082F812F82958F7070
:104DD0006CE0A0DB8F258295807FF026F82AF50114
:104DE000F082E394F9E0EF1609F0B0CFDD24EE2471
:104DF000CC24C394F3011081DD2021F40FE0F02EC8
:104E0000F12207C0F12EF2941FE0F1220894611CF8
:104E1000711C0881802F8F7062E07CDB182F802F3F
:104E200082958F7064E076DB8F258295807F1F25C9
:104E3000812B8883F4010081802F8F7068E06ADB0A
:104E4000182F802F82958F7063E064DB8F25829509
:104E5000807F1F25812BF4018083F5011081812F34
:104E60008F7066E057DB082F812F82958F706CE082
:104E700051DB9F2D98279295907FF0269F29F50171
:104E80009083E394F6E0EF1611F0DC24B3CF898130
:104E9000982B8881892BDF91CF911F910F91FF90E3
:104EA000EF90DF90CF90BF90AF909F908F907F90CA
:104EB0006F905F904F903F9008952F923F924F9246
:104EC0005F926F927F928F929F92AF92BF92CF929A
:104ED000DF92EF92FF920F931F93CF93DF93EC013A
:104EE0002B01E880CE2CC294BFE0CB2219818C2DFF
:104EF00090E02E2D30E02F703070822B932B212FDD
:104F000030E02F703070822B932B892B11F480E0CE
:104F1000DDC0AFE08A2E8122DA80FFE06F2E6D20A7
:104F2000882D662DF7DAA82E912E9294EFE09E221E
:104F3000892D2DDBA8268C2D692DECDA382E882DB5
:104F400026DB282E38268C2D662DE4DAF82E882DC7
:104F5000692DE0DA082F7FE0B72EBE208B2D6A2D59
:104F6000D9DA182F882D632DD5DA782E802F8F254A
:104F70006C2DD0DA7126782609F475C08C2D6A2D37
:104F8000C9DAE82E8C2D03DB0D2D02950F70602FF2
:104F9000C1DA182F8B2D692D462DC6DAF82E8B2DF0
:104FA000682D402FC1DA082F822D692DB3DA1E2516
:104FB0001F2510278127672DD6DAF20181936F0113
:104FC00009816FE0962E9022892D6A2DA3DA882E12
:104FD000F880AF2CA2945FE0A52202950F70BA80F2
:104FE0004FE0E42EEB208A2D602F4E2D9DDA182FF6
:104FF000FFE0FF226B2C62943FE063228F2D602F35
:10500000462D92DAB82E8E2DC2DA6F2D83DA082F54
:105010008A2D692D462D88DA18251B251027812712
:10502000672DA1DAF20181831A81812F82958F7019
:10503000632D70DAF82E812F8F70A9DA682F88819E
:1050400082958F7067DA082F198112951F70812F52
:105050009EDA612F5FDA0F258027672D84DAF6014B
:10506000818383E033C0AA2019F1862D90DA182FAE
:105070008D2D82958F70692D4DDA81276A2D73DA17
:10508000F2018083F9801A81612F62956F708F2DF4
:105090008F7040DA082F1F708F2D82958F70612FCF
:1050A00039DA80276A2D5FDAF201818382E00EC04F
:1050B0008C2D6B2D58DA182F882D6C2D54DAF201B7
:1050C0008083181711F08FEF01C081E0DF91CF913D
:1050D0001F910F91FF90EF90DF90CF90BF90AF9016
:1050E0009F908F907F906F905F904F903F902F9008
:1050F0000895BF92CF92DF92EF92FF920F931F938A
:10510000CF93DF93EC016A01623039F1633009F02B
:1051100040C0BB24EE248E2D1FDAF82E38DA182F6B
:105120006F2DF8D9082F812F6881F4D9182F8F2D72
:105130006981F0D9102718278A81181721F4F60100
:10514000F1926F01B394F2E0FB1520F0E3948FE04D
:10515000E81609F78B2D835020C0EE24FF248F2DF5
:10516000FBD9082F14DA182F802F6981D3D918277B
:105170008881181739F4F60101936F01E394F1E087
:10518000FE1520F0F3948FE0F81649F78E2D82502B
:1051900004C08881FA01808380E0DF91CF911F9164
:1051A0000F91FF90EF90DF90CF90BF9008954F92B6
:1051B0005F926F927F928F929F92AF92BF92CF92A7
:1051C000DF92EF92FF920F931F93CF93DF933C01F7
:1051D000EB012901423009F4B8C0FC01A080433042
:1051E00009F0E6C0FA80E9806E2D6F258F2D92D9E7
:1051F000982E6E2D8FD9082F1881812FC8D9682F2E
:10520000802F88D9612F86D9D82E6E2D61278E2DBB
:1052100081D9612F7FD9082F8F2DB9D9C82E802F22
:105220006C2D78D96F2D76D9B82E6F2D6127812FEF
:1052300071D96F2D6FD9182F8E2DA9D9082F812FD5
:10524000602F68D96E2D66D9BD24B8261FE0D12EF7
:10525000DA208F2D6D2D5ED91A2D12951F70612FBA
:1052600068278F2D57D9A82E802F6E2D53D9682FE0
:105270008A2D50D9082F8E2D6D2D4CD918278E2DA3
:10528000612F48D9882E8C2D6F2D44D9682F882DF9
:1052900041D9182FF30161816F70892D4E2D44D9AA
:1052A000102781276B2D5FD9F20181936F0108814F
:1052B000802F6DD9602F2ED9682F8A2D2BD9E82EFB
:1052C000F3011081612F6F70802F24D912951F7008
:1052D0001827802F612F1ED9982E1A81812F57D918
:1052E000612F18D9692D16D9F82EF30181818F709D
:1052F000602F10D9A82E0127812F602F0BD9682F7E
:105300008A2D08D9FE248F256B2D2DD9F20181839A
:10531000F8808F2D3CD96F2DFDD8682DFBD8E82E55
:105320001981812F34D9612FF5D8692DF3D8082F31
:10533000F126812F6F2DEED8682F8A2DEBD80E2500
:1053400080276B2D10D9F60131C01881812F1FD90C
:10535000D82EF9808F2D1BD9082F8D2D6F2DDAD8DF
:10536000E82E802F612FD6D8E826F3011081812FF7
:105370008F70602FCFD8082F812F82958F706F2D5F
:10538000C9D880276E2DEFD8F2018083F3011081F8
:10539000812F8F706D2DBED8082F812F82958F7031
:1053A0006881B8D880276E2DDED8F201818306C0CF
:1053B0008A2D8F706881D7D8F2018083DF91CF91D9
:1053C0001F910F91FF90EF90DF90CF90BF90AF9023
:1053D0009F908F907F906F905F904F9008955F9215
:1053E0006F927F928F929F92AF92BF92CF92DF92F5
:1053F000EF92FF920F931F93DF93CF93CDB7DEB75A
:105400002C970FB6F894DEBF0FBECDBF5C01842E83
:10541000022FDE011196E6E0F1E083E001900D92AB
:105420008150E1F7C501482D7E010894E11CF11C73
:1054300097016ADC882319F400E010E064C024E0DE
:10544000C22ED12CCC0EDD1EC701B60136DD982E42
:105450008FEF981619F40FEF10E055C08E01065F1C
:105460001F4FC601692DA80144DE882319F00EEFF5
:1054700010E049C097E0692E712C6C0E7D1EC701AB
:10548000B801492D930193DE6801730100E010E03B
:105490008EE0582E34C0F601808157D8F52DF81BC8
:1054A0008F2F880D8A30A8F4282F2695F701908138
:1054B00080FF09C0F501E20FF11D9295907F808178
:1054C0009827908306C0F501E20FF11D808189279E
:1054D0008083F701408198E020E030E0892F842329
:1054E00011F00F5F1F4F96952F5F3F4F243031050E
:1054F000A9F70894E11CF11C0894C11CD11C8E2D45
:105500008619891540F2C8012C960FB6F894DEBFB3
:105510000FBECDBFCF91DF911F910F91FF90EF9004
:10552000DF90CF90BF90AF909F908F907F906F90C3
:105530005F900895CF92DF92FF920F931F93CF93C6
:10554000DF936B018C01FF24C0E0D0E0B6016C0F4B
:105550007D1FC80140E028E042DF843040F4F80EAF
:105560000C5F1F4F2396CF30D10581F78F2DDF9130
:10557000CF911F910F91FF90DF90CF900895AF9240
:10558000BF92CF92DF92EF92FF920F931F93CF9330
:10559000DF935C01EB01142FFF24DD24EE2400E0F7
:1055A000CC24C39426C08F2D90E06D2D70E0153073
:1055B00050F06C0F7D1F8A0D9B1D402F29E00FDFDF
:1055C0001450101B0AC06C0F7D1F110F101B8A0D89
:1055D0009B1D402F212F03DF10E0843018F03EEF99
:1055E000E32E09C0F00E94E0F90E0C2593E0D90EDD
:1055F000E80E1123C1F68E2DDF91CF911F910F91EF
:10560000FF90EF90DF90CF90BF90AF900895CF9331
:10561000DF93EC01A0E040E050E0FA01EE5FF14FD3
:105620007491FE01E40FF51F8081782761E020E08E
:1056300030E0862F872309F0AF5F660F2F5F3F4F63
:1056400028303105B1F74F5F5F4F4430510529F7DE
:10565000A83008F4A0E08A2FDF91CF910895862723
:10566000282F22952827022E269526952025022EC2
:10567000269520252770082E892F26950794279593
:10568000902D822706942795902582270895FB0167
:10569000DC018D9181341CF08B350CF4805E6591BA
:1056A00061341CF06B350CF4605E861B611189F36C
:1056B000990B0895FB01DC010D900020E9F711978B
:1056C00005900D920020E1F70895FB01DC010590A3
:1056D0000D920020E1F70895FB01DC01415050409C
:1056E00048F005900D920020C9F701C01D9241506D
:1056F0005040E0F70895FB01DC0102C001900D92DB
:1057000041505040D8F70895DC0101C06D934150DD
:105710005040E0F70895FB01DC0101900D9200205C
:10572000E1F70895FB01DC014150504088F08D9174
:1057300081341CF08B350CF4805E619161341CF077
:105740006B350CF4605E861B611171F3990B089543
:10575000881BFCCFFB01DC014150504048F0019018
:105760000D920020C9F701C01D9241505040E0F752
:105770000895A0E0B0E0EEEBFBE2B9C07C01EB01E4
:105780008A01690109C0CE012196F6010995F70148
:1057900081937F010150104001151105A1F7CDB78C
:1057A000DEB7E8E0C0C0A0E0B0E0E8EDFBE29FC0FB
:1057B000EC017B018A01690109C0CE012196F70144
:1057C00061917F01F6010995015010400115110505
:1057D000A1F7CDB7DEB7E8E0A6C0FB019F01E894D2
:1057E0004230BCF04532ACF44A3029F497FB1EF449
:1057F000909581959F4F642F77271ED0805D8A33C7
:105800000CF0895D8193CB010097A9F716F45DE256
:1058100051931082C90100C0DC01FC01672F719116
:105820007723E1F7329704C07C916D937083629186
:10583000AE17BF07C8F30895AA1BBB1B51E107C0F1
:10584000AA1FBB1FA617B70710F0A61BB70B881F10
:10585000991F5A95A9F780959095BC01CD0108959F
:1058600097FB092E07260AD077FD04D0E5DF06D086
:1058700000201AF4709561957F4F0895F6F7909582
:1058800081959F4F0895A1E21A2EAA1BBB1BFD0113
:105890000DC0AA1FBB1FEE1FFF1FA217B307E4070F
:1058A000F50720F0A21BB30BE40BF50B661F771F67
:1058B000881F991F1A9469F7609570958095909547
:1058C0009B01AC01BD01CF0108959111089581564E
:1058D0008A5108F48052855808952F923F924F9232
:1058E0005F926F927F928F929F92AF92BF92CF9270
:1058F000DF92EF92FF920F931F93CF93DF93CDB779
:10590000DEB7CA1BDB0B0FB6F894DEBF0FBECDBFF0
:1059100009942A88398848885F846E847D848C84C1
:105920009B84AA84B984C884DF80EE80FD800C81CA
:105930001B81AA81B981CE0FD11D0FB6F894DEBFAD
:0C5940000FBECDBFED010895F894FFCF1D
:0A594C0078783A7878000000000037
:00000001FF
